:1000000061C07CC07CC07AC079C078C077C076C03F
:1000100075C074C073C07DC071C070C06FC06EC049
:100020006DC01502495E6473382FD0C78C9BA1B692
:10003000FDEA0111001122312A730011000126B3DB
:100040000233C4514475667776774655045D66760B
:1000500066772011049122232233085100132233A2
:10006000233344554454267F64775455445566578A
:10007000E673C8918A99AABBAABA88B9089DBABB87
:10008000AABBCCCDCCDDCEFFEA7FCCDDCDDDE6BF9B
:10009000EEFD889998992ABFAA9B88988899A8BB51
:1000A000EAB3CCDFC49DEFFFEEFFC85DECDDEEFFF1
:1000B000EEEFD780ACC281CAC19420982AC600E076
:1000C00000C8F7C411241FBECFE5D1E0DEBFCDBF0D
:1000D00010E0A0E6B0E0E6EFF5E003C0C895319689
:1000E0000D92A236B107D1F710E0A2E6B0E001C050
:1000F0001D92A436B107E1F716D07CC281CF1F92C2
:100100000F920FB60F9211240F900FBE0F901F90F9
:1001100018951F920F920FB60F9211240F900FBED9
:100120000F901F901895A0EFBFEF50D2802D282F71
:100130003327822F81508C3010F420936000DD240F
:10014000FF2410E0EE2401C01DE080916300992798
:1001500083709070892B99F5FF2089F5112379F52B
:1001600080E888B983E88BBB18BA8CED8ABBC89B42
:100170001CC081E092E8EFD08FE080B980E385BFBA
:1001800090E19BBF83E082BB9ABF7894DF9A889509
:10019000F8941BBE89E192E8DED082EE94E00197EC
:1001A000F1F7F5D080E090E0D6D080E285BF8BE01B
:1001B00080B981E088BF89BF83E083BF7894889548
:1001C00029B32095809163002827237059F089B3C3
:1001D000992783709070892B19F43EEFE32E6CC041
:1001E000EE246AC0DA9411F000E001C000E8EE20CD
:1001F00009F45FC0EA9409F05CC0DB9A81E092E800
:10020000AAD050916000952F8AE08895C9994EC078
:100210008150D9F7DA9A8AE08895C99947C0815008
:10022000D9F7DA98915081F760916300889549B3C6
:10023000409546274370242F3327862F9927809592
:1002400090958170907028233923232B51F05C30D6
:1002500009F47EC05F5FDA9A513011F01AE001C0F4
:100260001EE1862F842380FD04C0112321F011504C
:1002700011F4DA9810E06427C99BD8CF509360003E
:1002800060936300C89B11C0A0EFBFEF052EA6D1FD
:1002900081E88093640080E3809365008091600032
:1002A0008093660084E690E007D100E08BB3837F03
:1002B0008BBB002359F0202F80916300822780930D
:1002C00063009DE3D92E84E0F82E02C0FF20B1F137
:1002D00081E28093640080E38093650080916300F5
:1002E0008093660084E690E0E7D080E090E033D031
:1002F00092B7CD9B11C084E690E019D1882381F498
:1003000080916400803161F480916500833041F414
:10031000DB98DA9A13E00AC082B7891B863948F362
:10032000DB9ADA98FA9409F00FCF1EE089E192E89F
:1003300012D082EE94E00197F1F7FF24112309F423
:1003400004CF115009F001CF8BB3837F8BBBFDCE5F
:10035000DA9A51E085CFDF9820E197FF02C0DE9A5C
:1003600001C0DE98DC9A880F991FCD998160DC98D6
:10037000215099F7DF9ADF980895809160009927BE
:100380006AE370E011D185569B45E5DF0895CF9370
:10039000DF93C0E0D0E0E0E0F0E0EE0FFF1FEE54AE
:1003A000FF4FC895802D3196C895902DD4DF2196AA
:1003B000FD2FEC2FC930D10581F7DFDFDF91CF9121
:1003C000089581E89AECC7DF83E89AECC4DF0895CA
:1003D000CD9BFECF9927986BBEDF0895CD9BFECFB6
:1003E00080E090EBB8DF992708950F931F93CF9388
:1003F000DF93CDB7DEB721970FB6F894DEBF0FBEFF
:10040000CDBF982F80916200892738E02CE880FBCF
:1004100086950EF482273A95D1F780936200892F52
:1004200082958F7002E210E0F12FE02FE80FF11DAE
:10043000C895802D9983CCDF99819F70090F111D7C
:10044000F12FE02FC895802DC3DF21960FB6F894C9
:10045000DEBF0FBECDBFDF91CF911F910F910895E9
:10046000E82FE695FF27EE5CFF4FC895902D80FDA5
:1004700002C0892F03C0892F82958F7099278F70B2
:10048000907008951F93AADFEBDF182F1295107F4D
:10049000A5DFE6DF182B80916200812728E09CE829
:1004A00080FB86950EF489272A95D1F78093620008
:1004B000812F99271F910895EF92FF921F93CF9359
:1004C000DF93E82EF92E8AEA98EB45DF8AEA98EB6B
:1004D00042DF88E792E83FDF8AEA7ADF8DE278DF61
:1004E00084ED76DF10926200FF2DEE2D10811F70DB
:1004F000DF2DCE2D899179DF1F5F9F2D8E2D810FEE
:10050000911D11500196C817D907A1F7809162007B
:100510006CDF8AEA5DDFCD9BFECF89ED92E81BDFC1
:1005200050DFDF91CF911F91FF90EF900895CF9210
:10053000DF92FF920F931F93CF93DF93C82ED92E94
:10054000109262009FDF082F182F1F70DD2DCC2D19
:100550000993F090620096DF082F1F5F9D2D8C2D70
:10056000810F911D11500196C817D90789F729DF0E
:10057000F0268F2D9927DF91CF911F910F91FF903A
:10058000DF90CF900895CD9903C020E030E009C0FE
:1005900084E690E0CCDF20E030E0882311F421E015
:1005A00030E0932F822F08955527002480FF02C04A
:1005B000060E571F660F771F6115710521F096957E
:1005C0008795009799F7952F802D0895E199FECF93
:1005D000BFBBAEBBE09A11960DB20895E199FECF74
:1005E000BFBBAEBB0DBA11960FB6F894E29AE19A72
:0605F0000FBE0895FFCFCD
:0205F600030000
:00000001FF
